:1008DE005479706520616E79206B65797320746F21
:1008EE0020657869740A0054657374696E67200018
:1008FE000A00323030342053696C612052657365C2
:10090E006172636820436F2E2C4C74642E0A00446F
:10091E00323053514320537570657220514320502D
:10092E00726F6772616D2076312E320A00537065D8
:10093E006564203D2025640A000A4D61696E204DD4
:10094E00656E75202E2E2E0A0A002D2D2D2D205669
:10095E002D43343035314D202D2D2D2D0A00312EC5
:10096E002032304220506F72740A00322E203342F1
:10097E0020506F72740A00332E203142202620340C
:10098E0038352D4C454420506F72740A00342E2099
:10099E004F70746F2D496E7075740A00352E20538A
:1009AE006F756E6420262052656C61790A00362EB2
:1009BE00204F6E2D426F617264204B6579730A0071
:1009CE00372E20525443204453313330370A0038E7
:1009DE002E20454570726F6D2032344C4330340AF0
:1009EE00002D2D2D2D20562D43323035314D202DFD
:1009FE002D2D2D0A00432E2052656C617920262064
:100A0E00536F756E640A00442E20334220506F726D
:100A1E00740A00452E2031422026203438352D4CC4
:100A2E00454420506F72740A00462E2050434220D7
:100A3E0031302C31312C33322C33330A000A5365CA
:100A4E006C656374203A000A0A0032304220706FDF
:100A5E00727420284D41583733303029207769740D
:100A6E00682045582D4C4544202E2E2E0033422012
:100A7E00506F72742077697468204C50202E2E2E81
:100A8E000A00314220506F72742026203438352DE2
:100A9E004C45442077697468204C50202E2E2E0A27
:100AAE00004F70746F2D496E707574202E2E2E0AA5
:100ABE0000494E2D3120004F4B0A00494E2D322059
:100ACE00005479706520616E79206B6579730A0028
:100ADE00536F756E6420262052656C6179202E2E20
:100AEE002E0A004F6E2D426F617264204B65797332
:100AFE00202E2E2E0A0053572D31200053572D3203
:100B0E00200052544320445331333037202E2E2EA2
:100B1E000A0074696D652025303262783A253032CC
:100B2E0062783A253032627820206461746520251F
:100B3E00303262782F25303262782F25303262784B
:100B4E000A00454570726F6D2032344C43303420AC
:100B5E002E2E2E0A004572726F7220210A005479D1
:100B6E00706520616E79206B6579200052656C612D
:100B7E0079202E2E2E0A005043422031302C313156
:100B8E002C33322C33332077697468204C50202E4E
:040B9E002E2E0A00ED
:10000300EF4E60147D737C00ED1D70011CED4C7090
:09001300F7EF1F70011E80E822C6
:10001C00D3ED9400EC648094804022C2B57E01EE56
:10002C00D39F5008ED1D70011C0E80F3D2B57E01DC
:0E003C00EED39F50DBED1D70011C0E80F322F1
:0A004A007F0F7D107C2712001C229E
:0900540000000000000000002281
:06005D00D29112005422B2
:06006300C29112005422BC
:0E006900D290D291C290120054C291D2902235
:0A007700C290D291120054D29022E0
:10008100AB07AA067D01EB339202A2029290EB2507
:10009100E0FBEA33FA12005D1200630DBD09E7D2FD
:0E00A1009012005DA2909202120063A2022251
:1000AF00E4FF7E0112005DA2909202EF25E0FFA215
:1000BF0002E43342071200630EBE09E8D290120029
:1000CF005DA2909202120063A202B350027FFF2240
:1000DF008C228D23A9071200697FA07E0012008158
:1000EF00AF01120081AF23AE221200811200777F81
:0700FF00057E001200032240
:10010600AC071200697FA07E00120081AF041200C6
:10011600811200777F011200031200697FA17E0021
:100126001200811200AFAB071200777F017E00122A
:050136000003AF0322ED
:10013B008C248D258A268B27EF25E0541E4480FFC7
:10014B001200697E00120081AF25AE24120081AF30
:0A015B0027AE261200811200772261
:10016500A9077D047C00E4FBFA12013BAF017D0683
:10017500E4FBFA12013BAF017D097B557A001201C0
:100185003BAF017D0A7B557A0012013BAF017D0B28
:100195007B557A0012013BAF017D0C7B557A00122D
:1001A500013BAF017D0D7B557A0012013BAF017D0F
:1001B5000E7B557A0012013BAF017D0F7B557A000E
:0F01C50012013BAF017D047B017A0012013B2246
:1001D4008C248D25EF25E0541E4480FF1200697E97
:1001E400001200817F4C120081AF25AE24120081E1
:0401F400120077225C
:1001F8008C248D25EF25E0541E4480FF1200697E73
:10020800001200817F54120081AF25AE24120081B4
:040218001200772237
:10021C008C248D25EF25E0541E4480FF1200697E4E
:10022C00001200817F5C120081E525540FFF120043
:05023C00811200772291
:06024100D29112005422CC
:06024700C29112005422D6
:0E024D00D290D291C290120054C291D290224F
:0A025B00C290D291120054D29022FA
:10026500AB07AA067D01EB339201A2019290EB2523
:10027500E0FBEA33FA1202411202470DBD09E7D24B
:0E02850090120241A2909201120247A20122A1
:10029300E4FF7E01120241A2909201EF25E0FFA24A
:1002A30001E43342071202470EBE09E8D29012025C
:1002B30041A2909201120247A201B350027FFF2292
:1002C300E4FF7E01120241A2909201EF25E0FFA21A
:1002D30001E43342071202470EBE09E8C29012023C
:0702E30041120247D29022F4
:0A02EA0053087F530ABF530FEC22A4
:1002F40012024D7FD07E00120265E4FF120265E413
:10030400FC74082CF8E6FF7E001202650CBC08F1B0
:0403140012025B2254
:1003180012024D7FD07E00120265E4FF12026512C0
:10032800025B12005412024D7FD1120265E4FD12E5
:1003380002C3AC0774082DF8A6040DBD07F112021C
:07034800938F0F12025B22EC
:0A034F007BFF7A0879DE120C9E2273
:0A0359007BFF7A0879F5120C9E2252
:10036300758910E4F58DF58BC28E20B0FDD28EA277
:10037300B0B340FBC28EAF8DAD077C00ED7D00FCBA
:10038300AF8BEFFDE4759852758920D3ED9448EC5B
:10039300940D40097C047DB0758DE88040D3ED94C5
:1003A300A4EC940640097C097D60758DF4802ED3FE
:1003B300ED945CEC940340097C127DC0758DFA804A
:1003C3001CD3ED94AEEC940140097C257D80758DA2
:1003D300FD800A7C4B7D00758DFD438780D28EAEF8
:0403E30004AF05223C
:1003E7001203638E238F247522017BFF7A0879FE1F
:1003F700120C9E0522E522D3941440EE7BFF7A0966
:100407007900120C9E7BFF7A09791D120C9E7BFFE7
:0E0417007A09793B852328852429120C9E2220
:1004250012004A7BFF7A097947120C9E7BFF7A09F5
:100435007958120C9E7BFF7A09796C120C9E7BFF12
:100445007A097979120C9E7BFF7A097985120C9EBF
:100455007BFF7A09799B120C9E7BFF7A0979AA1298
:100465000C9E7BFF7A0979BC120C9E7BFF7A097979
:10047500CE120C9E7BFF7A0979DD120C9E7BFF7AEA
:100485000979EF120C9E7BFF7A0A7903120C9E7B89
:10049500FF7A0A7915120C9E7BFF7A0A7921120CD4
:1004A5009E7BFF7A0A7937120C9E7BFF7A0A794B7D
:1004B500120C9E120F8F120FA08F22E522C39431CA
:1004C5004007E522D394384014E522C394435003F2
:1004D500020428E522D3944640030204287BFF7AD0
:0904E5000A7955120C9EAF222287
:1004EE001203597BFF7A0A7958120C9EE4FF12010F
:1004FE00657901752301752201E4FFE523FD7C007A
:10050E001201D4E4FFE523FD1201F8E4FFE523FD1B
:10051E0012021C7F907E01120003E52325E0F523D5
:10052E000522E522D3940840D009B904C6752201EC
:10053E00752355E4FFE523FD7C001201D4E4FFE5AD
:10054E0023FD1201F8E4FFE523FD12021C7F587E05
:10055E00021200037523AAE4FFE523FD7C001201BD
:10056E00D4E4FFE523FD1201F8E4FFE523FD1202BA
:10057E001C7F587E021200030522E522D39403400D
:10058E00AFE4F523FFE523FD7C001201D4E4FFE583
:0E059E0023FD1201F8E4FFE523FD12021C22EA
:1005AC001203597BFF7A0A797B120C9E12034FA21D
:1005BC0098B35023E4F522E522D3940750F1E522B9
:1005CC00C43354E0FB441FF5907FC87E0012000337
:0E05DC002098DC052280E04390E0120F8F2271
:1005EA001203597BFF7A0A7990120C9E12034FA2CA
:1005FA0098B3501CC2B4C2B77FC87E001200032051
:10060A00980ED2B4D2B77FC87E001200033098DFAA
:08061A00D2B4D2B7120F8F22F7
:100622001203597BFF7A0A79AF120C9E7BFF7A0A7A
:1006320079BF120C9E20B2FD7BFF7A0A79C5120C9B
:100642009E7BFF7A0A79C9120C9E20B3FD7BFF7A4A
:100652000A79C5120C9E7BFF7A0A79CF120C9E1280
:030662000F8F22D5
:100665001203597BFF7A0A79DE120C9E12034FA200
:1006750098B3502AC2927F287D887C1312001C7F74
:10068500207E03120003209815D2927F467D407C80
:100695001F12001C7F207E031200033098D1D292D6
:0406A500120F8F227F
:1006A9001203597BFF7A0A79F1120C9E7BFF7A0BB0
:1006B9007904120C9E2093FD7BFF7A0A79C5120CEE
:1006C9009E7BFF7A0B790A120C9E2094FD7BFF7AA0
:1006D9000A79C5120C9E7BFF7A0A79CF120C9E12F9
:0306E9000F8F224E
:1006EC001203597BFF7A0B7910120C9E7508557505
:1006FC000959750A23750C28750D02750E04120222
:10070C00EA1202F4E508640560307F647E00120092
:10071C0003120318E508652260EA7BFF7A0B792047
:10072C00850A2885092985082A850C2B850D2C8599
:0B073C000E2D120C9E85082280CA22A0
:100747001203597BFF7A0B7950120C9EE4FF7DAAA6
:10075700FC1200DF7F017D557C001200DFC201E43F
:10076700FF120106EF64AA6002D2017F011201069F
:10077700EF64556002D20130010B7BFF7A0B79637E
:10078700120C9E80097BFF7A0A79C5120C9E7BFFAB
:0B0797007A0B796C120C9E120F8F225F
:1007A2001203597BFF7A0B797A120C9E12034FA225
:1007B20098B35063C2927F467D407C1F12001C7F1B
:1007C200207E0312000320984ED2927F207E0312D5
:1007D2000003209842C2937F3C7D407C1F12001C84
:1007E2007F207E0312000320982DD2937F207E0368
:1007F200120003209821C2947F327D407C1F120098
:100802001C7F207E0312000320980CD2947F207E4E
:1008120003120003309898D292D293D294120F8F7F
:0108220022B3
:100823001203597BFF7A0B7985120C9E12034FE456
:10083300FBA298B35032EB30E004D2908002C29016
:10084300EB30E104D2918002C291EB30E204D2B2E8
:100853008002C2B2EB30E304D2B38002C2B30B7F97
:0C0863000A7E0012000380C9120F8F22D1
:10086F001203E7120425EF120BAE08A13108A632CE
:10087F0008AB3308B03408B53508BA3608BF3708A7
:10088F00C43808C94308CE4408D34508D8460000E9
:10089F0008721204EE80CC1205AC80C71205EA80F4
:1008AF00C212062280BD12066580B81206A980B357
:1008BF001206EC80AE12074780A91207A280A4127D
:0F08CF0005AC809F1205EA809A120823809522BB
:03000000020BA24E
:0C0BA200787FE4F6D8FD75813802086FFA
:100BAE00D083D082F8E4937012740193700DA3A3D6
:100BBE0093F8740193F5828883E4737402936860EA
:060BCE00EFA3A3A380DFEA
:100C3C00E5342428F8E60534227825300902782892
:100C4C00E475F001120C2C020BD42002EB7F2ED297
:100C5C00028018EF540F2490D43440D4FF30060B8C
:100C6C00EF24BFB41A0050032461FFE53560021570
:100C7C00350538E5387002053730090D7825E475EF
:100C8C00F001120C2CEF020C1A020FB87403D209EB
:100C9C008003E4C209F5348B258A268927E4F535CF
:100CAC00F537F538E53560077F20120C7780F5F5C0
:100CBC0036C203C202C204C205C207C208C20A126B
:100CCC000C45FF700D3009057F00120C88AF38AE53
:100CDC003722B42561C2D5C206120C45FF24D0B40C
:100CEC000A00501C75F00A20D50DC535A42535F524
:100CFC00357002D20580E0C536A42536F53680D78E
:100D0C0024CFB41A00EF5004C2E5D206020E81D2F1
:100D1C000380C4D20280BED20480BAD2D580B8D2AD
:100D2C000780B27F20120C772004077401B53500C0
:100D3C0040F1120C3CFF120C77020CB0D20AD20814
:100D4C008093120C3CFB120C3CFA120C3CF94A4BF3
:100D5C007006794D7A0F7BFF200433E535602FAF99
:100D6C0036BF00011F7E008E82758300120BED6072
:100D7C00050EEE6F70F1C2D5EBC0E0EAC0E0E9C041
:100D8C00E0EE120EC5D0E0F9D0E0FAD0E0FB120B89
:100D9C00D4FF60A5EBC0E0EAC0E0E9C0E0120C773C
:100DAC00D0E02401F9D0E03400FAD0E0FBE5366065
:100DBC00DDD536DA80837BFF7A0E79C1D204809838
:100DCC00791080027908C208C20A8008D2D5790A43
:100DDC008004790AC2D5E4FAFDFEFF120C3CFC7BC0
:100DEC0008200313120C3CFD7B1030020A120C3C41
:100DFC00FE120C3CFF7B20EC3382D592D55013C3F2
:100E0C00E43002069FFFE49EFEE42003039DFDE414
:100E1C009CFCE4CBF8C203EC700CCFCECDCCE82418
:100E2C00F8F870F38017C3EF33FFEE33FEED33FDAC
:100E3C00EC33FCEB33FB994002FB0FD8E9EB3003AE
:100E4C0005F8D0E0C448B203C0E00AEC4D4E4F7830
:100E5C00207B0070C2EAC0E0120EC7D0F0D0E020B8
:100E6C000304C4C0E0C4B203C0F0120C60D0F0D5CF
:100E7C00F0EB020CB0120BAE0D4E530DCC580D1FF7
:100E8C004C0D1B420DD04F0DD8440DD8490D344399
:100E9C000DDE550DC2460DC2450DC2470F70500DEB
:100EAC00232D0D272E0D4A2B0D2B230D48200F5BC8
:100EBC002A00000D423F3F3F00790AA2D5200514BD
:100ECC00300709B910020404B9080104A2D520089E
:090EDC0002500104200466920496
:100EE500B535005032C0E07F203005177F30A204B1
:100EF50072087207500D120F1CC204C208C2077F88
:100F050030800F300703E9C0E0120C77300703D0BB
:100F1500E0F9D0E0B535CE3007177F30B9100C12A7
:100F25000C777F583006077F788003B90803120CC9
:100F3500773004057F2D020C777F20200AF87F2B60
:100F45002008F322920480CF286E756C6C29002D41
:100F550050434958D203120C3C3003F8C20378358C
:100F650030D504D2027836F6020CE1120C3C24038B
:100F7500B405004001E4900F5493120C68743A12C2
:0A0F85000C68D205753504020DCC8E
:100F8F0010000B120FDFBF0D027F0A020FB8AF1058
:010F9F00222F
:100FA000CEEFCEEEC39461400BEEC3947B5005EEC2
:080FB00024E0FF22CFEECF2266
:100BD400BB010689828A83E0225002E722BBFE021F
:090BE400E32289828A83E4932252
:100BED00BB010CE58229F582E5833AF583E02250BD
:100BFD0006E92582F8E622BBFE06E92582F8E22207
:0D0C0D00E58229F582E5833AF583E4932220
:100C1A00BB010689828A83F0225002F722BBFE01B9
:020C2A00F322B3
:100C2C00FAE6FB0808E6F925F0F618E6CA3AF622C9
:100FB800EFB40A07740D120FC3740A309811A89978
:100FC800B8130CC2983098FDA899C298B811F63099
:070FD80099FDC299F5992271
:0A0FDF003098FDAF99C2987E002201
:00000001FF
